:0200000480007A
:100000006F008004732F2034930F80006308FF0378
:10001000930F90006304FF03930FB0006300FF038E
:10002000130F000063040F0067000F00732F2034CC
:1000300063540F006F00400093E19153171F0000BD
:1000400023223FFC6FF09FFF93000000130100008C
:10005000930100001302000093020000130300004C
:100060009303000013040000930400001305000034
:10007000930500001306000093060000130700001C
:100080009307000013080000930800001309000004
:1000900093090000130A0000930A0000130B0000EC
:1000A000930B0000130C0000930C0000130D0000D4
:1000B000930D0000130E0000930E0000130F0000BC
:1000C000930F0000732540F16310050097020000B4
:1000D000938202017390523073500018970200000F
:1000E00093824202739052309B021000939252030B
:1000F0009382F2FF7390023B9302F0017390023AF5
:100100007350403097020000938242017390523046
:10011000735020307350303093010000970200007C
:10012000938282EE73905230130510001315F5017F
:10013000635C05000F00F00F930110009308D005D9
:10014000130500007300000093020000638A0200A0
:1001500073905210B7B200009B82921073902230BD
:100160007350003097020000938242017390123462
:10017000732540F1730020309300400113016000AB
:100180003BD720029303300093012000631A770CC1
:100190009B001000939000029380C0FE130160004A
:1001A0003BD72002B7B3AA2A9B8373AA93013000DE
:1001B0006318770A930040011301A0FF3BD7200288
:1001C0009303000093014000631C77089300C0FE76
:1001D0001301A0FF3BD720029303000093015000BE
:1001E00063107708B7000080130110003BD720028E
:1001F000B70300809301600063147706B7000080A6
:100200001301F0FF3BD7200293030000930170001D
:1002100063187704B7000080130100003BD7200269
:100220009303F0FF93018000631C7702930010009A
:10023000130100003BD720029303F0FF93019000CD
:100240006310770293000000130100003BD72002E7
:100250009303F0FF9301A000631477006310300252
:100260000F00F00F638001009391110093E11100E2
:100270009308D00513850100730000000F00F00FF4
:10028000930110009308D0051305000073000000CF
:10029000731000C00000000000000000000000001B
:1002A000000000000000000000000000000000004E
:0C02B00000000000000000000000000042
:1010000000000000000000000000000000000000E0
:1010100000000000000000000000000000000000D0
:1010200000000000000000000000000000000000C0
:1010300000000000000000000000000000000000B0
:081040000000000000000000A8
:040000058000000077
:00000001FF
